 GetProcessorInfo

 Timestamp is 1a2c74a6 (reproducible build file hash)

 Preferred load address is 0000000140000000

 Start         Length     Name                   Class
 0001:00000000 00000f60H .text$mn                CODE
 0001:00000f60 00000036H .text$mn$00             CODE
 0001:00000f96 00000036H .text$x                 CODE
 0002:00000000 000001d8H .idata$5                DATA
 0002:000001d8 00000038H .00cfg                  DATA
 0002:00000210 00000008H .CRT$XCA                DATA
 0002:00000218 00000008H .CRT$XCAA               DATA
 0002:00000220 00000008H .CRT$XCZ                DATA
 0002:00000228 00000008H .CRT$XIA                DATA
 0002:00000230 00000008H .CRT$XIAA               DATA
 0002:00000238 00000008H .CRT$XIAC               DATA
 0002:00000240 00000008H .CRT$XIZ                DATA
 0002:00000248 00000008H .CRT$XPA                DATA
 0002:00000250 00000008H .CRT$XPZ                DATA
 0002:00000258 00000008H .CRT$XTA                DATA
 0002:00000260 00000010H .CRT$XTZ                DATA
 0002:00000268 00000000H .gehcont$y              DATA
 0002:00000268 00000000H .gfids$y                DATA
 0002:00000270 00000390H .rdata                  DATA
 0002:00000600 00000000H .rdata$CastGuardVftablesA DATA
 0002:00000600 00000000H .rdata$CastGuardVftablesC DATA
 0002:00000600 0000005cH .rdata$voltmd           DATA
 0002:0000065c 000002ccH .rdata$zzzdbg           DATA
 0002:00000928 00000008H .rtc$IAA                DATA
 0002:00000930 00000008H .rtc$IZZ                DATA
 0002:00000938 00000008H .rtc$TAA                DATA
 0002:00000940 00000008H .rtc$TZZ                DATA
 0002:00000948 0000010cH .xdata                  DATA
 0002:00000a54 00000000H .edata                  DATA
 0002:00000a54 0000008cH .idata$2                DATA
 0002:00000ae0 00000018H .idata$3                DATA
 0002:00000af8 000001d8H .idata$4                DATA
 0002:00000cd0 000004e2H .idata$6                DATA
 0003:00000000 00000040H .data                   DATA
 0003:00000040 000005f8H .bss                    DATA
 0004:00000000 0000018cH .pdata                  DATA

  Address         Publics by Value              Rva+Base               Lib:Object

 0000:00000000       __AbsoluteZero             0000000000000000     <absolute>
 0000:00000000       ___safe_se_handler_count   0000000000000000     <absolute>
 0000:00000000       ___safe_se_handler_table   0000000000000000     <absolute>
 0000:00000000       __arm64x_extra_rfe_table   0000000000000000     <absolute>
 0000:00000000       __arm64x_extra_rfe_table_size 0000000000000000     <absolute>
 0000:00000000       __arm64x_native_entrypoint 0000000000000000     <absolute>
 0000:00000000       __arm64x_redirection_metadata 0000000000000000     <absolute>
 0000:00000000       __arm64x_redirection_metadata_count 0000000000000000     <absolute>
 0000:00000000       __dynamic_value_reloc_table 0000000000000000     <absolute>
 0000:00000000       __enclave_config           0000000000000000     <absolute>
 0000:00000000       __guard_check_icall_a64n_fptr 0000000000000000     <absolute>
 0000:00000000       __guard_eh_cont_count      0000000000000000     <absolute>
 0000:00000000       __guard_eh_cont_table      0000000000000000     <absolute>
 0000:00000000       __guard_fids_count         0000000000000000     <absolute>
 0000:00000000       __guard_fids_table         0000000000000000     <absolute>
 0000:00000000       __guard_iat_count          0000000000000000     <absolute>
 0000:00000000       __guard_iat_table          0000000000000000     <absolute>
 0000:00000000       __guard_longjmp_count      0000000000000000     <absolute>
 0000:00000000       __guard_longjmp_table      0000000000000000     <absolute>
 0000:00000000       __hybrid_auxiliary_iat     0000000000000000     <absolute>
 0000:00000000       __hybrid_auxiliary_iat_copy 0000000000000000     <absolute>
 0000:00000000       __hybrid_code_map          0000000000000000     <absolute>
 0000:00000000       __hybrid_code_map_count    0000000000000000     <absolute>
 0000:00000000       __x64_code_ranges_to_entry_points 0000000000000000     <absolute>
 0000:00000000       __x64_code_ranges_to_entry_points_count 0000000000000000     <absolute>
 0000:00000100       __guard_flags              0000000000000100     <absolute>
 0000:00000000       __ImageBase                0000000140000000     <linker-defined>
 0001:00000000       __local_stdio_printf_options 0000000140001000 f i exeGetProcessorInfo.obj
 0001:00000008       main                       0000000140001008 f   exeGetProcessorInfo.obj
 0001:000001fc       printf                     00000001400011fc f i exeGetProcessorInfo.obj
 0001:00000250       __GSHandlerCheck           0000000140001250 f   MSVCRT:gshandler.obj
 0001:00000270       __GSHandlerCheckCommon     0000000140001270 f   MSVCRT:gshandler.obj
 0001:000002e0       __security_check_cookie    00000001400012e0 f   MSVCRT:amdsecgs.obj
 0001:00000560       mainCRTStartup             0000000140001560 f   MSVCRT:exe_main.obj
 0001:00000574       __raise_securityfailure    0000000140001574 f   MSVCRT:gs_report.obj
 0001:000005a8       __report_gsfailure         00000001400015a8 f   MSVCRT:gs_report.obj
 0001:000006f0       __scrt_acquire_startup_lock 00000001400016f0 f   MSVCRT:utility.obj
 0001:0000072c       __scrt_initialize_crt      000000014000172c f   MSVCRT:utility.obj
 0001:00000778       __scrt_initialize_onexit_tables 0000000140001778 f   MSVCRT:utility.obj
 0001:00000804       __scrt_is_nonwritable_in_current_image 0000000140001804 f   MSVCRT:utility.obj
 0001:0000089c       __scrt_release_startup_lock 000000014000189c f   MSVCRT:utility.obj
 0001:000008c0       __scrt_uninitialize_crt    00000001400018c0 f   MSVCRT:utility.obj
 0001:000008ec       _onexit                    00000001400018ec f   MSVCRT:utility.obj
 0001:00000928       atexit                     0000000140001928 f   MSVCRT:utility.obj
 0001:00000940       __security_init_cookie     0000000140001940 f   MSVCRT:gs_support.obj
 0001:000009ec       __scrt_exe_initialize_mta  00000001400019ec f   MSVCRT:utility_desktop.obj
 0001:000009ec       __scrt_initialize_winrt    00000001400019ec f   MSVCRT:utility_desktop.obj
 0001:000009ec       __scrt_stub_for_initialize_mta 00000001400019ec f   MSVCRT:utility_desktop.obj
 0001:000009ec       _get_startup_commit_mode   00000001400019ec f   MSVCRT:commit_mode.obj
 0001:000009ec       _get_startup_new_mode      00000001400019ec f   MSVCRT:new_mode.obj
 0001:000009ec       _get_startup_thread_locale_mode 00000001400019ec f   MSVCRT:thread_locale.obj
 0001:000009ec       _matherr                   00000001400019ec f   MSVCRT:matherr.obj
 0001:000009f0       _get_startup_argv_mode     00000001400019f0 f   MSVCRT:argv_mode.obj
 0001:000009f8       _get_startup_file_mode     00000001400019f8 f   MSVCRT:file_mode.obj
 0001:00000a00       ?__scrt_initialize_type_info@@YAXXZ 0000000140001a00 f   MSVCRT:tncleanup.obj
 0001:00000a10       __acrt_initialize          0000000140001a10 f   MSVCRT:ucrt_stubs.obj
 0001:00000a10       __acrt_uninitialize        0000000140001a10 f   MSVCRT:ucrt_stubs.obj
 0001:00000a10       __scrt_stub_for_acrt_initialize 0000000140001a10 f   MSVCRT:ucrt_stubs.obj
 0001:00000a10       __scrt_stub_for_acrt_uninitialize 0000000140001a10 f   MSVCRT:ucrt_stubs.obj
 0001:00000a10       __vcrt_initialize          0000000140001a10 f   MSVCRT:ucrt_stubs.obj
 0001:00000a10       __vcrt_uninitialize        0000000140001a10 f   MSVCRT:ucrt_stubs.obj
 0001:00000a10       _should_initialize_environment 0000000140001a10 f   MSVCRT:env_mode.obj
 0001:00000a14       _guard_check_icall_nop     0000000140001a14 f   MSVCRT:guard_support.obj
 0001:00000a14       _initialize_denormal_control 0000000140001a14 f   MSVCRT:denormal_control.obj
 0001:00000a14       _initialize_invalid_parameter_handler 0000000140001a14 f   MSVCRT:invalid_parameter_handler.obj
 0001:00000a18       __local_stdio_scanf_options 0000000140001a18 f i MSVCRT:default_local_stdio_options.obj
 0001:00000a20       __scrt_initialize_default_local_stdio_options 0000000140001a20 f   MSVCRT:default_local_stdio_options.obj
 0001:00000a3c       __scrt_is_user_matherr_present 0000000140001a3c f   MSVCRT:matherr_detection.obj
 0001:00000a48       __scrt_get_dyn_tls_init_callback 0000000140001a48 f   MSVCRT:dyn_tls_init.obj
 0001:00000a50       __scrt_get_dyn_tls_dtor_callback 0000000140001a50 f   MSVCRT:dyn_tls_dtor.obj
 0001:00000a58       __crt_debugger_hook        0000000140001a58 f   MSVCRT:utility_desktop.obj
 0001:00000a60       __scrt_fastfail            0000000140001a60 f   MSVCRT:utility_desktop.obj
 0001:00000bac       __scrt_initialize_mta      0000000140001bac f   MSVCRT:utility_desktop.obj
 0001:00000bb4       __scrt_is_managed_app      0000000140001bb4 f   MSVCRT:utility_desktop.obj
 0001:00000c08       __scrt_set_unhandled_exception_filter 0000000140001c08 f   MSVCRT:utility_desktop.obj
 0001:00000c18       __scrt_unhandled_exception_filter 0000000140001c18 f   MSVCRT:utility_desktop.obj
 0001:00000c74       _RTC_Initialize            0000000140001c74 f   MSVCRT:initsect.obj
 0001:00000cb0       _RTC_Terminate             0000000140001cb0 f   MSVCRT:initsect.obj
 0001:00000cec       __isa_available_init       0000000140001cec f   MSVCRT:cpu_disp.obj
 0001:00000e98       __scrt_is_ucrt_dll_in_use  0000000140001e98 f   MSVCRT:ucrt_detection.obj
 0001:00000eb0       memset                     0000000140001eb0 f   vcruntime:VCRUNTIME140.dll
 0001:00000eb6       __C_specific_handler       0000000140001eb6 f   vcruntime:VCRUNTIME140.dll
 0001:00000ebc       __current_exception        0000000140001ebc f   vcruntime:VCRUNTIME140.dll
 0001:00000ec2       __current_exception_context 0000000140001ec2 f   vcruntime:VCRUNTIME140.dll
 0001:00000ec8       _seh_filter_exe            0000000140001ec8 f   ucrt:api-ms-win-crt-runtime-l1-1-0.dll
 0001:00000ece       _set_app_type              0000000140001ece f   ucrt:api-ms-win-crt-runtime-l1-1-0.dll
 0001:00000ed4       __setusermatherr           0000000140001ed4 f   ucrt:api-ms-win-crt-math-l1-1-0.dll
 0001:00000eda       _configure_narrow_argv     0000000140001eda f   ucrt:api-ms-win-crt-runtime-l1-1-0.dll
 0001:00000ee0       _initialize_narrow_environment 0000000140001ee0 f   ucrt:api-ms-win-crt-runtime-l1-1-0.dll
 0001:00000ee6       _get_initial_narrow_environment 0000000140001ee6 f   ucrt:api-ms-win-crt-runtime-l1-1-0.dll
 0001:00000eec       _initterm                  0000000140001eec f   ucrt:api-ms-win-crt-runtime-l1-1-0.dll
 0001:00000ef2       _initterm_e                0000000140001ef2 f   ucrt:api-ms-win-crt-runtime-l1-1-0.dll
 0001:00000ef8       exit                       0000000140001ef8 f   ucrt:api-ms-win-crt-runtime-l1-1-0.dll
 0001:00000efe       _exit                      0000000140001efe f   ucrt:api-ms-win-crt-runtime-l1-1-0.dll
 0001:00000f04       _set_fmode                 0000000140001f04 f   ucrt:api-ms-win-crt-stdio-l1-1-0.dll
 0001:00000f0a       __p___argc                 0000000140001f0a f   ucrt:api-ms-win-crt-runtime-l1-1-0.dll
 0001:00000f10       __p___argv                 0000000140001f10 f   ucrt:api-ms-win-crt-runtime-l1-1-0.dll
 0001:00000f16       _cexit                     0000000140001f16 f   ucrt:api-ms-win-crt-runtime-l1-1-0.dll
 0001:00000f1c       _c_exit                    0000000140001f1c f   ucrt:api-ms-win-crt-runtime-l1-1-0.dll
 0001:00000f22       _register_thread_local_exe_atexit_callback 0000000140001f22 f   ucrt:api-ms-win-crt-runtime-l1-1-0.dll
 0001:00000f28       _configthreadlocale        0000000140001f28 f   ucrt:api-ms-win-crt-locale-l1-1-0.dll
 0001:00000f2e       _set_new_mode              0000000140001f2e f   ucrt:api-ms-win-crt-heap-l1-1-0.dll
 0001:00000f34       __p__commode               0000000140001f34 f   ucrt:api-ms-win-crt-stdio-l1-1-0.dll
 0001:00000f3a       _initialize_onexit_table   0000000140001f3a f   ucrt:api-ms-win-crt-runtime-l1-1-0.dll
 0001:00000f40       _register_onexit_function  0000000140001f40 f   ucrt:api-ms-win-crt-runtime-l1-1-0.dll
 0001:00000f46       _crt_atexit                0000000140001f46 f   ucrt:api-ms-win-crt-runtime-l1-1-0.dll
 0001:00000f4c       terminate                  0000000140001f4c f   ucrt:api-ms-win-crt-runtime-l1-1-0.dll
 0001:00000f52       memcpy                     0000000140001f52 f   vcruntime:VCRUNTIME140.dll
 0001:00000f70       _guard_dispatch_icall_nop  0000000140001f70 f   MSVCRT:guard_dispatch.obj
 0001:00000f90       _guard_xfg_dispatch_icall_nop 0000000140001f90 f   MSVCRT:guard_xfg_dispatch.obj
 0002:00000000       __imp_VerSetConditionMask  0000000140002000     kernel32:KERNEL32.dll
 0002:00000008       __imp_GetLastError         0000000140002008     kernel32:KERNEL32.dll
 0002:00000010       __imp_GetCurrentProcess    0000000140002010     kernel32:KERNEL32.dll
 0002:00000018       __imp_GetProcessGroupAffinity 0000000140002018     kernel32:KERNEL32.dll
 0002:00000020       __imp_VerifyVersionInfoW   0000000140002020     kernel32:KERNEL32.dll
 0002:00000028       __imp_GetActiveProcessorCount 0000000140002028     kernel32:KERNEL32.dll
 0002:00000030       __imp_RtlCaptureContext    0000000140002030     kernel32:KERNEL32.dll
 0002:00000038       __imp_RtlLookupFunctionEntry 0000000140002038     kernel32:KERNEL32.dll
 0002:00000040       __imp_RtlVirtualUnwind     0000000140002040     kernel32:KERNEL32.dll
 0002:00000048       __imp_UnhandledExceptionFilter 0000000140002048     kernel32:KERNEL32.dll
 0002:00000050       __imp_SetUnhandledExceptionFilter 0000000140002050     kernel32:KERNEL32.dll
 0002:00000058       __imp_TerminateProcess     0000000140002058     kernel32:KERNEL32.dll
 0002:00000060       __imp_IsProcessorFeaturePresent 0000000140002060     kernel32:KERNEL32.dll
 0002:00000068       __imp_QueryPerformanceCounter 0000000140002068     kernel32:KERNEL32.dll
 0002:00000070       __imp_GetCurrentProcessId  0000000140002070     kernel32:KERNEL32.dll
 0002:00000078       __imp_GetCurrentThreadId   0000000140002078     kernel32:KERNEL32.dll
 0002:00000080       __imp_GetSystemTimeAsFileTime 0000000140002080     kernel32:KERNEL32.dll
 0002:00000088       __imp_InitializeSListHead  0000000140002088     kernel32:KERNEL32.dll
 0002:00000090       __imp_IsDebuggerPresent    0000000140002090     kernel32:KERNEL32.dll
 0002:00000098       __imp_GetModuleHandleW     0000000140002098     kernel32:KERNEL32.dll
 0002:000000a0       \177KERNEL32_NULL_THUNK_DATA 00000001400020a0     kernel32:KERNEL32.dll
 0002:000000a8       __imp_memset               00000001400020a8     vcruntime:VCRUNTIME140.dll
 0002:000000b0       __imp___C_specific_handler 00000001400020b0     vcruntime:VCRUNTIME140.dll
 0002:000000b8       __imp___current_exception  00000001400020b8     vcruntime:VCRUNTIME140.dll
 0002:000000c0       __imp___current_exception_context 00000001400020c0     vcruntime:VCRUNTIME140.dll
 0002:000000c8       __imp_memcpy               00000001400020c8     vcruntime:VCRUNTIME140.dll
 0002:000000d0       \177VCRUNTIME140_NULL_THUNK_DATA 00000001400020d0     vcruntime:VCRUNTIME140.dll
 0002:000000d8       __imp__set_new_mode        00000001400020d8     ucrt:api-ms-win-crt-heap-l1-1-0.dll
 0002:000000e0       __imp_malloc               00000001400020e0     ucrt:api-ms-win-crt-heap-l1-1-0.dll
 0002:000000e8       __imp_free                 00000001400020e8     ucrt:api-ms-win-crt-heap-l1-1-0.dll
 0002:000000f0       \177api-ms-win-crt-heap-l1-1-0_NULL_THUNK_DATA 00000001400020f0     ucrt:api-ms-win-crt-heap-l1-1-0.dll
 0002:000000f8       __imp__configthreadlocale  00000001400020f8     ucrt:api-ms-win-crt-locale-l1-1-0.dll
 0002:00000100       \177api-ms-win-crt-locale-l1-1-0_NULL_THUNK_DATA 0000000140002100     ucrt:api-ms-win-crt-locale-l1-1-0.dll
 0002:00000108       __imp___setusermatherr     0000000140002108     ucrt:api-ms-win-crt-math-l1-1-0.dll
 0002:00000110       \177api-ms-win-crt-math-l1-1-0_NULL_THUNK_DATA 0000000140002110     ucrt:api-ms-win-crt-math-l1-1-0.dll
 0002:00000118       __imp__get_initial_narrow_environment 0000000140002118     ucrt:api-ms-win-crt-runtime-l1-1-0.dll
 0002:00000120       __imp__initterm            0000000140002120     ucrt:api-ms-win-crt-runtime-l1-1-0.dll
 0002:00000128       __imp__initialize_narrow_environment 0000000140002128     ucrt:api-ms-win-crt-runtime-l1-1-0.dll
 0002:00000130       __imp__configure_narrow_argv 0000000140002130     ucrt:api-ms-win-crt-runtime-l1-1-0.dll
 0002:00000138       __imp__exit                0000000140002138     ucrt:api-ms-win-crt-runtime-l1-1-0.dll
 0002:00000140       __imp__set_app_type        0000000140002140     ucrt:api-ms-win-crt-runtime-l1-1-0.dll
 0002:00000148       __imp___p___argc           0000000140002148     ucrt:api-ms-win-crt-runtime-l1-1-0.dll
 0002:00000150       __imp___p___argv           0000000140002150     ucrt:api-ms-win-crt-runtime-l1-1-0.dll
 0002:00000158       __imp__cexit               0000000140002158     ucrt:api-ms-win-crt-runtime-l1-1-0.dll
 0002:00000160       __imp__c_exit              0000000140002160     ucrt:api-ms-win-crt-runtime-l1-1-0.dll
 0002:00000168       __imp__register_thread_local_exe_atexit_callback 0000000140002168     ucrt:api-ms-win-crt-runtime-l1-1-0.dll
 0002:00000170       __imp_exit                 0000000140002170     ucrt:api-ms-win-crt-runtime-l1-1-0.dll
 0002:00000178       __imp__initterm_e          0000000140002178     ucrt:api-ms-win-crt-runtime-l1-1-0.dll
 0002:00000180       __imp_terminate            0000000140002180     ucrt:api-ms-win-crt-runtime-l1-1-0.dll
 0002:00000188       __imp__initialize_onexit_table 0000000140002188     ucrt:api-ms-win-crt-runtime-l1-1-0.dll
 0002:00000190       __imp__register_onexit_function 0000000140002190     ucrt:api-ms-win-crt-runtime-l1-1-0.dll
 0002:00000198       __imp__crt_atexit          0000000140002198     ucrt:api-ms-win-crt-runtime-l1-1-0.dll
 0002:000001a0       __imp__seh_filter_exe      00000001400021a0     ucrt:api-ms-win-crt-runtime-l1-1-0.dll
 0002:000001a8       \177api-ms-win-crt-runtime-l1-1-0_NULL_THUNK_DATA 00000001400021a8     ucrt:api-ms-win-crt-runtime-l1-1-0.dll
 0002:000001b0       __imp__set_fmode           00000001400021b0     ucrt:api-ms-win-crt-stdio-l1-1-0.dll
 0002:000001b8       __imp___stdio_common_vfprintf 00000001400021b8     ucrt:api-ms-win-crt-stdio-l1-1-0.dll
 0002:000001c0       __imp___acrt_iob_func      00000001400021c0     ucrt:api-ms-win-crt-stdio-l1-1-0.dll
 0002:000001c8       __imp___p__commode         00000001400021c8     ucrt:api-ms-win-crt-stdio-l1-1-0.dll
 0002:000001d0       \177api-ms-win-crt-stdio-l1-1-0_NULL_THUNK_DATA 00000001400021d0     ucrt:api-ms-win-crt-stdio-l1-1-0.dll
 0002:000001d8       __guard_check_icall_fptr   00000001400021d8     MSVCRT:guard_support.obj
 0002:000001e0       __guard_xfg_check_icall_fptr 00000001400021e0     MSVCRT:guard_support.obj
 0002:000001e8       __guard_dispatch_icall_fptr 00000001400021e8     MSVCRT:guard_support.obj
 0002:000001f0       __guard_xfg_dispatch_icall_fptr 00000001400021f0     MSVCRT:guard_support.obj
 0002:000001f8       __guard_xfg_table_dispatch_icall_fptr 00000001400021f8     MSVCRT:guard_support.obj
 0002:00000200       __castguard_check_failure_os_handled_fptr 0000000140002200     MSVCRT:guard_support.obj
 0002:00000208       __guard_memcpy_fptr        0000000140002208     vcruntime:softmemtag.obj
 0002:00000210       __xc_a                     0000000140002210     MSVCRT:initializers.obj
 0002:00000220       __xc_z                     0000000140002220     MSVCRT:initializers.obj
 0002:00000228       __xi_a                     0000000140002228     MSVCRT:initializers.obj
 0002:00000240       __xi_z                     0000000140002240     MSVCRT:initializers.obj
 0002:00000248       __xp_a                     0000000140002248     MSVCRT:initializers.obj
 0002:00000250       __xp_z                     0000000140002250     MSVCRT:initializers.obj
 0002:00000258       __xt_a                     0000000140002258     MSVCRT:initializers.obj
 0002:00000260       __xt_z                     0000000140002260     MSVCRT:initializers.obj
 0002:00000270       ??_C@_0CP@JHDDEBLJ@GetActiveProcessorCount?5failed?5@ 0000000140002270     exeGetProcessorInfo.obj
 0002:000002a0       ??_C@_0BF@GEBMGLHG@IsWindowsServer?3?5?$CFd?6@ 00000001400022a0     exeGetProcessorInfo.obj
 0002:000002b8       ??_C@_0DI@LMKJHEG@Active?5processor?5count?5across?5a@ 00000001400022b8     exeGetProcessorInfo.obj
 0002:000002f0       ??_C@_0DL@NMDIJEKG@Unexpected?5group?5count?5of?50?5fro@ 00000001400022f0     exeGetProcessorInfo.obj
 0002:00000330       ??_C@_0DE@IPLNLFFH@Unexpected?5GetProcessGroupAffin@ 0000000140002330     exeGetProcessorInfo.obj
 0002:00000368       ??_C@_0BA@EJMMBNFL@malloc?5failed?4?6@ 0000000140002368     exeGetProcessorInfo.obj
 0002:00000378       ??_C@_0BO@IFJIJCBL@Active?5processors?5per?5group?3?5@ 0000000140002378     exeGetProcessorInfo.obj
 0002:00000398       ??_C@_0DD@FEKPKFDI@GetActiveProcessorCount?$CI?$CFd?$CJ?5fai@ 0000000140002398     exeGetProcessorInfo.obj
 0002:000003cc       ??_C@_03DPLIHHLN@?$CFd?0@  00000001400023cc     exeGetProcessorInfo.obj
 0002:000003e0       __xmm@ffffffffffffffffffffffffffffffff 00000001400023e0     MSVCRT:utility.obj
 0002:000003f0       _load_config_used          00000001400023f0     MSVCRT:loadcfg.obj
 0002:00000600       __volatile_metadata        0000000140002600     <linker-defined>
 0002:00000928       __rtc_iaa                  0000000140002928     MSVCRT:initsect.obj
 0002:00000930       __rtc_izz                  0000000140002930     MSVCRT:initsect.obj
 0002:00000938       __rtc_taa                  0000000140002938     MSVCRT:initsect.obj
 0002:00000940       __rtc_tzz                  0000000140002940     MSVCRT:initsect.obj
 0002:00000a54       __IMPORT_DESCRIPTOR_KERNEL32 0000000140002a54     kernel32:KERNEL32.dll
 0002:00000a68       __IMPORT_DESCRIPTOR_VCRUNTIME140 0000000140002a68     vcruntime:VCRUNTIME140.dll
 0002:00000a7c       __IMPORT_DESCRIPTOR_api-ms-win-crt-heap-l1-1-0 0000000140002a7c     ucrt:api-ms-win-crt-heap-l1-1-0.dll
 0002:00000a90       __IMPORT_DESCRIPTOR_api-ms-win-crt-stdio-l1-1-0 0000000140002a90     ucrt:api-ms-win-crt-stdio-l1-1-0.dll
 0002:00000aa4       __IMPORT_DESCRIPTOR_api-ms-win-crt-runtime-l1-1-0 0000000140002aa4     ucrt:api-ms-win-crt-runtime-l1-1-0.dll
 0002:00000ab8       __IMPORT_DESCRIPTOR_api-ms-win-crt-math-l1-1-0 0000000140002ab8     ucrt:api-ms-win-crt-math-l1-1-0.dll
 0002:00000acc       __IMPORT_DESCRIPTOR_api-ms-win-crt-locale-l1-1-0 0000000140002acc     ucrt:api-ms-win-crt-locale-l1-1-0.dll
 0002:00000ae0       __NULL_IMPORT_DESCRIPTOR   0000000140002ae0     kernel32:KERNEL32.dll
 0003:00000000       __security_cookie          0000000140004000     MSVCRT:gs_cookie.obj
 0003:00000008       __security_cookie_complement 0000000140004008     MSVCRT:gs_cookie.obj
 0003:00000010       __scrt_native_dllmain_reason 0000000140004010     MSVCRT:utility.obj
 0003:00000014       __scrt_default_matherr     0000000140004014     MSVCRT:matherr.obj
 0003:00000018       __isa_available            0000000140004018     MSVCRT:cpu_disp.obj
 0003:0000001c       __isa_enabled              000000014000401c     MSVCRT:cpu_disp.obj
 0003:00000020       __memset_fast_string_threshold 0000000140004020     MSVCRT:cpu_disp.obj
 0003:00000028       __memset_nt_threshold      0000000140004028     MSVCRT:cpu_disp.obj
 0003:00000030       __scrt_ucrt_dll_is_in_use  0000000140004030     MSVCRT:ucrt_stubs.obj
 0003:000005b0       __scrt_current_native_startup_state 00000001400045b0     MSVCRT:utility.obj
 0003:000005b8       __scrt_native_startup_lock 00000001400045b8     MSVCRT:utility.obj
 0003:00000600       ?__type_info_root_node@@3U__type_info_node@@A 0000000140004600     MSVCRT:tncleanup.obj
 0003:00000610       ?_OptionsStorage@?1??__local_stdio_scanf_options@@9@4_KA 0000000140004610     MSVCRT:default_local_stdio_options.obj
 0003:00000618       __scrt_debugger_hook_flag  0000000140004618     MSVCRT:utility_desktop.obj
 0003:0000061c       __favor                    000000014000461c     MSVCRT:cpu_disp.obj
 0003:00000620       ?_OptionsStorage@?1??__local_stdio_printf_options@@9@9 0000000140004620     <common>
 0003:00000628       __dyn_tls_dtor_callback    0000000140004628     <common>
 0003:00000630       __dyn_tls_init_callback    0000000140004630     <common>

 entry point at        0001:00000560

 Static symbols

 0000:ffff9000       .debug$S                   0000000140000000     vcruntime:VCRUNTIME140.dll
 0000:ffff9000       .debug$S                   0000000140000000     vcruntime:VCRUNTIME140.dll
 0000:ffff9000       .debug$S                   0000000140000000     vcruntime:VCRUNTIME140.dll
 0000:ffff9000       .debug$S                   0000000140000000     vcruntime:VCRUNTIME140.dll
 0000:ffff9000       .debug$S                   0000000140000000     vcruntime:VCRUNTIME140.dll
 0000:ffff9000       .debug$S                   0000000140000000     vcruntime:VCRUNTIME140.dll
 0000:ffff9000       .debug$S                   0000000140000000     ucrt:api-ms-win-crt-heap-l1-1-0.dll
 0000:ffff9000       .debug$S                   0000000140000000     ucrt:api-ms-win-crt-heap-l1-1-0.dll
 0000:ffff9000       .debug$S                   0000000140000000     ucrt:api-ms-win-crt-heap-l1-1-0.dll
 0000:ffff9000       .debug$S                   0000000140000000     ucrt:api-ms-win-crt-locale-l1-1-0.dll
 0000:ffff9000       .debug$S                   0000000140000000     ucrt:api-ms-win-crt-math-l1-1-0.dll
 0000:ffff9000       .debug$S                   0000000140000000     ucrt:api-ms-win-crt-runtime-l1-1-0.dll
 0000:ffff9000       .debug$S                   0000000140000000     ucrt:api-ms-win-crt-runtime-l1-1-0.dll
 0000:ffff9000       .debug$S                   0000000140000000     ucrt:api-ms-win-crt-runtime-l1-1-0.dll
 0000:ffff9000       .debug$S                   0000000140000000     ucrt:api-ms-win-crt-runtime-l1-1-0.dll
 0000:ffff9000       .debug$S                   0000000140000000     ucrt:api-ms-win-crt-runtime-l1-1-0.dll
 0000:ffff9000       .debug$S                   0000000140000000     ucrt:api-ms-win-crt-runtime-l1-1-0.dll
 0000:ffff9000       .debug$S                   0000000140000000     ucrt:api-ms-win-crt-runtime-l1-1-0.dll
 0000:ffff9000       .debug$S                   0000000140000000     ucrt:api-ms-win-crt-runtime-l1-1-0.dll
 0000:ffff9000       .debug$S                   0000000140000000     ucrt:api-ms-win-crt-runtime-l1-1-0.dll
 0000:ffff9000       .debug$S                   0000000140000000     ucrt:api-ms-win-crt-runtime-l1-1-0.dll
 0000:ffff9000       .debug$S                   0000000140000000     ucrt:api-ms-win-crt-runtime-l1-1-0.dll
 0000:ffff9000       .debug$S                   0000000140000000     ucrt:api-ms-win-crt-runtime-l1-1-0.dll
 0000:ffff9000       .debug$S                   0000000140000000     ucrt:api-ms-win-crt-runtime-l1-1-0.dll
 0000:ffff9000       .debug$S                   0000000140000000     ucrt:api-ms-win-crt-runtime-l1-1-0.dll
 0000:ffff9000       .debug$S                   0000000140000000     ucrt:api-ms-win-crt-runtime-l1-1-0.dll
 0000:ffff9000       .debug$S                   0000000140000000     ucrt:api-ms-win-crt-runtime-l1-1-0.dll
 0000:ffff9000       .debug$S                   0000000140000000     ucrt:api-ms-win-crt-runtime-l1-1-0.dll
 0000:ffff9000       .debug$S                   0000000140000000     ucrt:api-ms-win-crt-runtime-l1-1-0.dll
 0000:ffff9000       .debug$S                   0000000140000000     ucrt:api-ms-win-crt-runtime-l1-1-0.dll
 0000:ffff9000       .debug$S                   0000000140000000     ucrt:api-ms-win-crt-runtime-l1-1-0.dll
 0000:ffff9000       .debug$S                   0000000140000000     ucrt:api-ms-win-crt-runtime-l1-1-0.dll
 0000:ffff9000       .debug$S                   0000000140000000     ucrt:api-ms-win-crt-stdio-l1-1-0.dll
 0000:ffff9000       .debug$S                   0000000140000000     ucrt:api-ms-win-crt-stdio-l1-1-0.dll
 0000:ffff9000       .debug$S                   0000000140000000     ucrt:api-ms-win-crt-stdio-l1-1-0.dll
 0000:ffff9000       .debug$S                   0000000140000000     ucrt:api-ms-win-crt-stdio-l1-1-0.dll
 0000:ffff9000       .debug$S                   0000000140000000     kernel32:KERNEL32.dll
 0000:ffff9000       .debug$S                   0000000140000000     kernel32:KERNEL32.dll
 0000:ffff9000       .debug$S                   0000000140000000     kernel32:KERNEL32.dll
 0000:ffff9000       .debug$S                   0000000140000000     kernel32:KERNEL32.dll
 0000:ffff9000       .debug$S                   0000000140000000     kernel32:KERNEL32.dll
 0000:ffff9000       .debug$S                   0000000140000000     kernel32:KERNEL32.dll
 0000:ffff9000       .debug$S                   0000000140000000     kernel32:KERNEL32.dll
 0000:ffff9000       .debug$S                   0000000140000000     kernel32:KERNEL32.dll
 0000:ffff9000       .debug$S                   0000000140000000     kernel32:KERNEL32.dll
 0000:ffff9000       .debug$S                   0000000140000000     kernel32:KERNEL32.dll
 0000:ffff9000       .debug$S                   0000000140000000     kernel32:KERNEL32.dll
 0000:ffff9000       .debug$S                   0000000140000000     kernel32:KERNEL32.dll
 0000:ffff9000       .debug$S                   0000000140000000     kernel32:KERNEL32.dll
 0000:ffff9000       .debug$S                   0000000140000000     kernel32:KERNEL32.dll
 0000:ffff9000       .debug$S                   0000000140000000     kernel32:KERNEL32.dll
 0000:ffff9000       .debug$S                   0000000140000000     kernel32:KERNEL32.dll
 0000:ffff9000       .debug$S                   0000000140000000     kernel32:KERNEL32.dll
 0000:ffff9000       .debug$S                   0000000140000000     kernel32:KERNEL32.dll
 0000:ffff9000       .debug$S                   0000000140000000     kernel32:KERNEL32.dll
 0000:ffff9000       .debug$S                   0000000140000000     kernel32:KERNEL32.dll
 0000:ffff9000       .debug$S                   0000000140000000     kernel32:KERNEL32.dll
 0001:000002d0       $$000000                   00000001400012d0     MSVCRT:amdsecgs.obj
 0001:00000300       ?pre_c_initialization@@YAHXZ 0000000140001300 f   MSVCRT:exe_main.obj
 0001:000003b8       ?post_pgo_initialization@@YAHXZ 00000001400013b8 f   MSVCRT:exe_main.obj
 0001:000003c8       ?pre_cpp_initialization@@YAXXZ 00000001400013c8 f   MSVCRT:exe_main.obj
 0001:000003e4       ?__scrt_common_main_seh@@YAHXZ 00000001400013e4 f   MSVCRT:exe_main.obj
 0001:0000067c       capture_previous_context   000000014000167c f   MSVCRT:gs_report.obj
 0001:00000f60       $$000000                   0000000140001f60     MSVCRT:guard_dispatch.obj
 0001:00000f80       $$000000                   0000000140001f80     MSVCRT:guard_xfg_dispatch.obj
 0001:00000f96       ?filt$0@?0??__scrt_common_main_seh@@YAHXZ@4HA 0000000140001f96 f   MSVCRT:exe_main.obj
 0001:00000fb4       __scrt_is_nonwritable_in_current_image$filt$0 0000000140001fb4 f   MSVCRT:utility.obj
 0002:00000218       ?pre_cpp_initializer@@3P6AXXZEA 0000000140002218     MSVCRT:exe_main.obj
 0002:00000230       ?pre_c_initializer@@3P6AHXZEA 0000000140002230     MSVCRT:exe_main.obj
 0002:00000238       ?post_pgo_initializer@@3P6AHXZEA 0000000140002238     MSVCRT:exe_main.obj
 0002:000003d0       GS_ExceptionPointers       00000001400023d0     MSVCRT:gs_report.obj
 0002:00000948       $unwind$printf             0000000140002948     exeGetProcessorInfo.obj
 0002:00000954       $unwind$main               0000000140002954     exeGetProcessorInfo.obj
 0002:00000978       $unwind$__GSHandlerCheckCommon 0000000140002978     MSVCRT:gshandler.obj
 0002:00000980       $unwind$__scrt_initialize_default_local_stdio_options 0000000140002980     MSVCRT:default_local_stdio_options.obj
 0002:00000980       $unwind$?post_pgo_initialization@@YAHXZ 0000000140002980     MSVCRT:exe_main.obj
 0002:00000980       $unwind$?pre_cpp_initialization@@YAXXZ 0000000140002980     MSVCRT:exe_main.obj
 0002:00000980       $unwind$mainCRTStartup     0000000140002980     MSVCRT:exe_main.obj
 0002:00000980       $unwind$__GSHandlerCheck   0000000140002980     MSVCRT:gshandler.obj
 0002:00000980       $unwind$__scrt_acquire_startup_lock 0000000140002980     MSVCRT:utility.obj
 0002:00000980       $unwind$atexit             0000000140002980     MSVCRT:utility.obj
 0002:00000980       $unwind$__scrt_is_managed_app 0000000140002980     MSVCRT:utility_desktop.obj
 0002:00000988       $xdatasym                  0000000140002988     MSVCRT:amdsecgs.obj
 0002:0000098c       $unwind$?pre_c_initialization@@YAHXZ 000000014000298c     MSVCRT:exe_main.obj
 0002:0000098c       $unwind$__raise_securityfailure 000000014000298c     MSVCRT:gs_report.obj
 0002:0000098c       $unwind$__scrt_initialize_crt 000000014000298c     MSVCRT:utility.obj
 0002:0000098c       $unwind$__scrt_initialize_onexit_tables 000000014000298c     MSVCRT:utility.obj
 0002:0000098c       $unwind$__scrt_release_startup_lock 000000014000298c     MSVCRT:utility.obj
 0002:0000098c       $unwind$__scrt_uninitialize_crt 000000014000298c     MSVCRT:utility.obj
 0002:0000098c       $unwind$_onexit            000000014000298c     MSVCRT:utility.obj
 0002:00000994       $unwind$?__scrt_common_main_seh@@YAHXZ 0000000140002994     MSVCRT:exe_main.obj
 0002:000009cc       $unwind$?filt$0@?0??__scrt_common_main_seh@@YAHXZ@4HA 00000001400029cc     MSVCRT:exe_main.obj
 0002:000009d4       $unwind$__report_gsfailure 00000001400029d4     MSVCRT:gs_report.obj
 0002:000009dc       $unwind$capture_previous_context 00000001400029dc     MSVCRT:gs_report.obj
 0002:000009e8       $unwind$__scrt_is_nonwritable_in_current_image 00000001400029e8     MSVCRT:utility.obj
 0002:00000a08       $unwind$__scrt_is_nonwritable_in_current_image$filt$0 0000000140002a08     MSVCRT:utility.obj
 0002:00000a10       $unwind$__security_init_cookie 0000000140002a10     MSVCRT:gs_support.obj
 0002:00000a1c       $unwind$__scrt_fastfail    0000000140002a1c     MSVCRT:utility_desktop.obj
 0002:00000a2c       $unwind$_RTC_Initialize    0000000140002a2c     MSVCRT:initsect.obj
 0002:00000a2c       $unwind$_RTC_Terminate     0000000140002a2c     MSVCRT:initsect.obj
 0002:00000a2c       $unwind$__scrt_unhandled_exception_filter 0000000140002a2c     MSVCRT:utility_desktop.obj
 0002:00000a38       $unwind$__isa_available_init 0000000140002a38     MSVCRT:cpu_disp.obj
 0002:00000a48       $xdatasym                  0000000140002a48     MSVCRT:guard_dispatch.obj
 0002:00000a50       $xdatasym                  0000000140002a50     MSVCRT:guard_xfg_dispatch.obj
 0002:00000e9e       .idata$6                   0000000140002e9e     kernel32:KERNEL32.dll
 0002:00000f02       .idata$6                   0000000140002f02     vcruntime:VCRUNTIME140.dll
 0002:00001104       .idata$6                   0000000140003104     ucrt:api-ms-win-crt-heap-l1-1-0.dll
 0002:00001124       .idata$6                   0000000140003124     ucrt:api-ms-win-crt-stdio-l1-1-0.dll
 0002:00001144       .idata$6                   0000000140003144     ucrt:api-ms-win-crt-runtime-l1-1-0.dll
 0002:00001166       .idata$6                   0000000140003166     ucrt:api-ms-win-crt-math-l1-1-0.dll
 0002:00001186       .idata$6                   0000000140003186     ucrt:api-ms-win-crt-locale-l1-1-0.dll
 0003:00000040       GS_ExceptionRecord         0000000140004040     MSVCRT:gs_report.obj
 0003:000000e0       GS_ContextRecord           00000001400040e0     MSVCRT:gs_report.obj
 0003:000005c0       ?is_initialized_as_dll@@3_NA 00000001400045c0     MSVCRT:utility.obj
 0003:000005c1       ?module_local_atexit_table_initialized@@3_NA 00000001400045c1     MSVCRT:utility.obj
 0003:000005c8       ?module_local_atexit_table@@3U_onexit_table_t@@A 00000001400045c8     MSVCRT:utility.obj
 0003:000005e0       ?module_local_at_quick_exit_table@@3U_onexit_table_t@@A 00000001400045e0     MSVCRT:utility.obj
